:061800000AEF0CF00102EA
:10180800FACF2CF0FBCF2DF0A2ED12F09BEF11F0E8
:0A18180028C408F535EC11F01200A9
:021826001000B0
:10191400A6A21200FDD700000E0E0E0E0E0E000041
:101924000E0E0E0E0E0ED6CF03F0D7CF04F003C06A
:1019340001F004C002F0120060C0A9FFA69CA69E9C
:10194400A68000F000F0A8501200D6CF62F0D7CFE6
:1019540063F062C060F063C061F0120035EC11F016
:10196400C00E8016FC0E84163F0E926E030E966E09
:10197400130ED36E12000001616F010E000100010D
:10198400F56F0001615160C055F001010101005182
:10199400120001507F0BD56E000ED76E000ED66E6E
:1019A400F29401AE02D0F28A01D0F29AD58E1200DE
:1019B400600ED36E030E0A6E200E096E0906D8A0BF
:1019C4000A060928D8B40A28D8A4F8D735EC11F0A7
:1019D4001200698468986D82010E476E000E156EC0
:1019E400750E146E000E176E000E166E000E196E34
:1019F400000E186E6CEC12F0120001C007F002C069
:101A040008F008D007C0D9FF08C0DAFF03C0DFFF21
:101A1400074A082A0506D8A006060528D8B40628C9
:101A2400D8B41200EFD7555000010001F55DD8A0DD
:101A340002D0000E0DD000010001F551010D01018D
:101A4400000EF324D96E0101010EF420DA6EDF508A
:101A54001200000E476E000E156E740E146E000E0A
:101A6400176E000E166E000E196E000E186E6CECDA
:101A740012F06D92699401D0689468A41200FCD7A6
:101A8400600ED36E030E00010001696F200E000189
:101A9400686F000100016807D8A069070001682980
:101AA400D8B46929D8A4F5D710EC14F0120004C0F6
:101AB40053F004C001F0CCEC13F0046E00010001FB
:101AC400F72B020E0001F76507D0056E000E00012A
:101AD4000001F76F055001D0049204501200000E6B
:101AE40000010001616F000E0001606F9EEC0CF0BC
:101AF40000010001EC6F040E00010001EC6508D048
:101B04000001626F000E00010001EC6F00016251E0
:101B140012000401040E00010001D86F0401280E14
:101B24000001D76F000E00010001DC6F080E0001F8
:101B3400DB6F180E00010001DE6F180E0001DD6F6F
:101B440000010001DA8F120000010001EE6716D0D7
:101B5400000E6D6E000E696E160E6F6E9F0E6B6E2C
:101B64007B0E696ED08EA28AA08AF28E01D06D8619
:101B74006DA6FDD7010E00010001EE6F120060C0DA
:101B840066F061C067F00BD066C0D9FF67C0DAFFAA
:101B9400000162C0DFFF00010001664B672B0001FA
:101BA40000016407D8A0650700016429D8B4652939
:101BB400D8B41200E9D70001000161516011D8A422
:101BC40002D0270E15D00001000161516011D8B474
:101BD4000ED00A0E00010001605D000E0001615983
:101BE400D8B005D00001000160511D0F01D02C0EAA
:101BF400120070A01BD0800E3CC0D9FF3DC0DAFF9C
:101C0400DF6213D0840EDFC0D9FFE0C0DAFFDF62E9
:101C14000CD03CC0D9FF3DC0DAFF0C0EDF6E3CC0D7
:101C2400D9FF3DC0DAFF000EDB8E7090689A120077
:101C340063C053F063C060F07AEC18F00001000157
:101C4400636F00010001F72B020E0001F76509D054
:101C54000001646F000E00010001F76F0001645180
:101C640003D00001000163930001000163511200DD
:101C740000010001F62B050E00010001F66508D0F5
:101C84000001686F000E00010001F66F0001685149
:101C94008AEC0CF0000E00010001616F020E0001DD
:101CA400606FF6C062F05DEC0FF095EC15F0120079
:101CB40000010001F32B050E00010001F36508D0BB
:101CC4000001686F000E00010001F36F000168510C
:101CD4008AEC0CF0000E00010001616F040E00019B
:101CE400606FF3C062F05DEC0FF0E7EC15F01200EA
:101CF40000010001EF2B040E00010001EF6508D084
:101D04000001686F000E00010001EF6F00016851CF
:101D14008AEC0CF0000E00010001616F030E00015B
:101D2400606FEFC062F05DEC0FF039EC16F012005A
:101D340000010001EC2B040E00010001EC6508D049
:101D44000001686F000E00010001EC6F0001685192
:101D54008AEC0CF0000E00010001616F000E00011E
:101D6400606FECC062F05DEC0FF08BEC16F01200CB
:101D740000010001F42B040E00010001F46508D0F9
:101D84000001686F000E00010001F46F000168514A
:101D94008AEC0CF0000E00010001616F010E0001DD
:101DA400606FF4C062F05DEC0FF0DDEC16F0120031
:101DB40000010001EB2B060E00010001EB6508D0C9
:101DC4000001686F000E00010001EB6F0001685113
:101DD4008AEC0CF0000E00010001616F050E000199
:101DE400606FEBC062F05DEC0FF081EC17F0120055
:101DF40000010001F12B030E00010001F16508D080
:101E04000001686F000E00010001F16F00016851CC
:101E14008AEC0CF0000E00010001616F060E000157
:101E2400606FF1C062F05DEC0FF02FEC17F0120060
:101E34000001606F010E00010001616F000160513B
:101E440000010001EC51030AD8B40ED000010001D6
:101E5400EC51040AD8B408D00001606F000E0001F0
:101E64000001616F00016051000100016151120025
:101E74000001D66F000E00010001696F0001D65108
:101E8400A3EC10F072EC27F0A6EC0DF0200E00018C
:101E94000001EE6101D0FAD76DA208D0A9EC0FF0D1
:101EA4000009D8B4F3D7F6EC0FF0F0D76DB2EED743
:101EB4008EEC33F0EBD70001636F000E00010001DC
:101EC400646F0001635160C0A9FF62C0A8FFA69EB1
:101ED400A69CA684000EF2BE010E00010001646FF0
:101EE400F29E550EA76EAA0EA76EA682A6B2FED7C4
:101EF4000001000164B102D0F29E01D0F28EA694DA
:101F040012000001626F000E00010001636F000106
:101F1400625100010001F251D8B415D060C0D9FF5C
:101F240061C0DAFFDF50DD0BD8A40DD00001000141
:101F3400F451D8B408D00001626F010E0001000111
:101F4400636F000162510001000163511200C00E71
:101F54008916FC0E8D16000E926E000E966E000110
:101F6400606F010E00010001616F00016051835038
:101F7400FF0AFC0BD8A40DD08150FF0A3F0BD8A454
:101F840008D00001606F000E00010001616F0001C4
:101F9400605100010001615112000CA408D00BC073
:101FA40001F00D6E000E026E0D5043EC15F00CA204
:101FB40008D00BC001F00D6E010E026E0D5043EC03
:101FC40015F00B50010D700EF3240D6E0F0EF4205E
:101FD4000E6E0DC00FF00EC010F00FC0D9FF10C070
:101FE400DAFF0CC0DFFF120000010001ED51D8B48C
:101FF40022D04750D8B41FD0A09A42EC0DF06D9275
:10200400000E476E0E0E3B6E100E3A6E3A06D8A0C6
:102014003B063B503A10D8A4F9D76D84070E3B6EAB
:10202400080E3A6E3A06D8A03B063B503A10D8A4A4
:10203400F9D76D94A08A1200800E00010001F561A9
:1020440012D000010001F551010D0101000EF3242D
:10205400D96E0101010EF420DA6E000162C0DFFFC7
:1020640000010001F52B800E00010001F5610ED086
:1020740000010001F551010D0101000EF324D96E98
:102084000101010EF420DA6E000EDF6E12004E50D4
:10209400020AD8A403D0D6EC21F025D0000E4E6E4F
:1020A40046661FD020EE01F03E50D9263F50DA227A
:1020B400080EDF6E20EE02F03E50D9263F50DA22A1
:1020C400200EDE6E040EDD6E3EC0D9FF3FC0DAFF87
:1020D4000C0EDF6E3EC0D9FF3FC0DAFF000EDB8E70
:1020E40002D0000E466E12000001656F000E000162
:1020F4000001676F00016551000107D068C062F0FC
:102104001EEC10F000010001672B00016751010D66
:10211400F3500001000163250001656FF4500001D4
:10212400000164210001666F65C0F6FF66C0F7FF19
:1021340008000001F5CF68F0000100016867DED7F0
:10214400120023D0000EBD6E000EBA6E0F0EC11227
:10215400C00E89163F0E926E93688A68F19E380EFF
:102164008B16C70E8B12380E946EFC0E8C16030E53
:102174008C12FC0E956EFC0E8C12848E8D948D84C4
:10218400030E966EBBEC1AF009D0000100016951F0
:10219400000AD8B4D7D7010AD8A4030A1200000150
:1021A40000016951000100016B03F3CF6DF0F4CF1E
:1021B4006EF0000100016951000100016C03F3CFCE
:1021C400F4FFF36AF350000100016D27F45000019D
:1021D40000016E23000100016A51000100016B033C
:1021E400F3CFF4FFF36AF350000100016D27F450BC
:1021F400000100016E236DC069F06EC06AF0120028
:1022040008C504F059EC0DF0076E07A007D0066E60
:10221400010E016E065002EC12F006D0066E010E9D
:10222400016E065037EC12F007A207D0066E020EBC
:10223400016E065002EC12F006D0066E020E016E1C
:10224400065037EC12F007A407D0066E030E016E99
:10225400065002EC12F006D0066E030E016E065014
:1022640037EC12F012006DA229D0086E010E016E37
:10227400085037EC12F0086E020E016E085037EC6D
:1022840012F0086E030E016E085037EC12F01DD0E8
:1022940002EC11F01AD0086E010E016E085002EC27
:1022A40012F0086E020E016E085002EC12F0086E75
:1022B400030E016E085002EC12F007D00001000179
:1022C400EE51200AD8B4E4D7E6D7120055500001E5
:1022D4000001F55DD8A00AD00001606F000E000176
:1022E4000001F56F00016051000E22D000010001D1
:1022F400F551010D0101000EF324D96E0101010E07
:10230400F420DA6EDF5000010001616F000100016A
:10231400F52B00010001616708D00001606F000E19
:1023240000010001F56F00016051000100016151DD
:10233400120001EE00F0C10EEE6AE806FDE100EEC7
:10234400D7F0270EEE6AE806FDE100EE3AF0250E1E
:10235400EE6AE806FDE11A0EF66E190EF76E000E2F
:10236400F86E01EEC1F010EE10F00900F5CFEEFFAB
:10237400E550E150FAE1040EF66E180EF76E000E09
:10238400F86E0900F5CFFEF00900F5CFFFF0000E5E
:10239400F86E00013AEF0FF071C077F072C078F078
:1023A4006FC075F070C076F01FD0000177C0F6FFE3
:1023B400000178C0F7FFF86A75C0D9FF76C0DAFF6C
:1023C400070EF76403D00800F55005D0F6CFE9FFF7
:1023D400F7CFEAFFEF50DF6E00010001774B782B57
:1023E40000010001754B762B000100017307D8A092
:1023F400740700017329D8B47429D8B41200D5D74E
:10240400FE0EF66E170EF76E0900F5CF02F0090006
:10241400F5CF03F0020E025C000E0358D8A002D0E0
:10242400010E01D0000E046E12D004B002D08C92C2
:1024340001D08C8219D004B002D08C9001D08C8051
:1024440013D004B002D08B9401D08B840DD00150F2
:10245400000AD8B409D0010AD8B4E7D7030AD8B41B
:10246400EAD7010AD8B4EDD71200FE0EF66E170EA5
:10247400F76E0900F5CF02F00900F5CF03F0020E64
:10248400025C000E0358D8B002D0010E01D0000E39
:10249400046E12D004B002D08C9201D08C8219D078
:1024A40004B002D08C9001D08C8013D004B002D040
:1024B4008B9401D08B840DD00150000AD8B409D07C
:1024C400010AD8B4E7D7030AD8B4EAD7010AD8B4C2
:1024D400EDD712000CD0B0EC0CF031D0DAEC0CF0EB
:1024E4002ED012EC13F02BD09EEC20F028D014C088
:1024F4001AF015C01BF01B50000AD8B404D07F0A90
:10250400D8B41BD01CD01A50010AD8B4EAD7030A95
:10251400D8B415D0010AD8B4E7D7060AD8B40FD076
:10252400770AD8B40CD0010AD8B409D0070AD8B4B1
:10253400D5D7010AD8B4CFD702D01A50FF0A120057
:102544000600E9CF2EF0EACF2FF0E1CF30F0E2CF52
:1025540031F0D9CF32F0DACF33F0F3CF34F0F4CF17
:1025640035F0F6CF36F0F7CF37F0F8CF38F0F5CFB7
:1025740039F0CEEC23F039C0F5FF38C0F8FF37C08E
:10258400F7FF36C0F6FF35C0F4FF34C0F3FF33C0A5
:10259400DAFF32C0D9FF31C0E2FF30C0E1FF2FC003
:1025A400EAFF2EC0E9FF2DC0FBFF2CC0FAFF11008B
:1025B40060C066F061C067F020D000010001665180
:1025C400F66EE96E070EEA6E000100016751EA64D7
:1025D40003D0EA6EEF5003D0F76E0800F550000107
:1025E40000016219D8A405D066C060F067C061F02C
:1025F40016D000010001664B672B0001000164073F
:10260400D8A0650700016429D8B46529D8A4D5D712
:10261400000E00010001616F000E0001606F1200E6
:10262400000E01010101816F000E0101806F000E97
:1026340005010501086F116E010E0B6E1150126E2B
:102644001E0E0C6E1250CFEC0FF0116E010E016EC7
:102654001150126E000E026E12500501050E046E2A
:102664000501080E036E136E010E056E1350EEEC99
:1026740019F001C082F102C083F1116E170E016ED0
:102684001150CBEC0CF095EC0CF001C042F002C000
:1026940043F01200FE0EF66E170EF76E0900F5CF2A
:1026A40061F00900F5CF62F0020E0001615D000ED9
:1026B4006259D8A002D0010E01D0000E0001000121
:1026C400636F18D00001000163B102D08C9201D075
:1026D4008C821FD00001000163B102D08C9001D024
:1026E4008C8017D00001000163B102D08B9401D01B
:1026F4008B840FD0000100016051000AD8B409D0C6
:10270400010AD8B4DFD7030AD8B4E4D7010AD8B48D
:10271400E9D71200FE0EF66E170EF76E0900F5CF1C
:1027240061F00900F5CF62F0020E0001615D000E58
:102734006259D8B002D0010E01D0000E0001000190
:10274400636F18D00001000163B102D08C9201D0F4
:102754008C821FD00001000163B102D08C9001D0A3
:102764008C8017D00001000163B102D08B9401D09A
:102774008B840FD0000100016051000AD8B409D045
:10278400010AD8B4DFD7030AD8B4E4D7010AD8B40D
:10279400E9D7120000010001F451D8A428D03CD09C
:1027A400EBC002F0010E036E022A02D0D890033669
:1027B400022EFCD70350FF0A0116EBC002F0F2C050
:1027C40003F0022A02D0D8900336022EFCD70CD094
:1027D400EBC002F0FD0E0226F2C003F0022A02D082
:1027E400D8900336022EFCD70350011215D00001F5
:1027F4000001EB51000AD8B4D3D7010AD8B4D0D71A
:10280400030AD8B4CDD7010AD8B4E2D7070AD8B49A
:10281400DFD7010AD8B4DCD7015012006DA241D031
:102824000001676F010E00010001606F0001675134
:102834008CEC13F00001676F020E00010001606F61
:10284400000167518CEC13F00001676F030E000167
:102854000001606F000167518CEC13F029D0D3ECB8
:1028640017F026D00001676F010E00010001606FB0
:10287400000167514CEC13F00001676F020E000178
:102884000001606F000167514CEC13F00001676FA9
:10289400030E00010001606F000167514CEC13F05E
:1028A40007D000010001EE51200AD8B4D8D7DAD7F6
:1028B4001200000E00010001616F010E0001606F43
:1028C4009EEC0CF000010001F46F040E0001000105
:1028D400F46508D00001626F000E00010001F46F7E
:1028E40000016251000E00010001616F050E00013C
:1028F400606F9EEC0CF000010001EB6F060E00010E
:102904000001EB6508D00001626F040E00010001B4
:10291400EB6F00016251000E00010001616F060EB1
:102924000001606F9EEC0CF000010001F16F030EDA
:1029340000010001F16508D00001626F000E000182
:102944000001F16F00016251120039D062C0D9FF59
:1029540063C0DAFFDF500001666F60C0D9FF61C059
:10296400DAFFDF5000016619D8B421D062C0D9FF64
:1029740063C0DAFFDF500001666F676B0001661FFA
:10298400671F664B672B60C0D9FF61C0DAFFDF5059
:102994000001686F00016851000166250001000113
:1029A400606F00010001000E6721616F1AD0000101
:1029B4000001604B612B00010001624B632B00019D
:1029C40000016407D8A0650700016429D8B465290B
:1029D400D8A4BCD7000E00010001616F000E0001F5
:1029E400606F1200000E566E000E4A6E000E486EA6
:1029F400000E496E000E466E000E4E6EDFC0D9FF0B
:102A0400E0C0DAFF7F0EDF16040E00010001DF1BB9
:102A1400DFC0D9FFE0C0DAFF7F0EDF16040E00012D
:102A24000001DF1B3EC0D9FF3FC0DAFF7F0EDF1677
:102A3400000E00010001FB6F000E00010001FD6F9C
:102A4400000E0001FC6F000E00010001DA6F000EA1
:102A540000010001DC6F000E0001DB6F75EC1EF05D
:102A6400000E156E030E146E000E176E000E166E19
:102A7400000E196E000E186E6CEC12F0FCEC1CF0DB
:102A840012000401040E0A6E0401000E096ED890AF
:102A94000234036E046A04360150056E066AD89047
:102AA40005360636D8900536063603500524076EDB
:102AB40004500620086ED89007360836D89007369A
:102AC40008360750092608500A2209C0D9FF0AC04F
:102AD400DAFF7F0EDF16026609D00150020D0001F5
:102AE400E30EF324D96E0001000E08D00150020D4C
:102AF4000001DF0EF324D96E0001000EF420DA6E1B
:102B040009C0DEFF0AC0DDFF09C0D9FF0AC0DAFF31
:102B1400BF0EDF1620EE04F00950D9260A50DA223F
:102B2400400EDF12120000010001F651050D0A0EDD
:102B3400F32400010001656F7F0EF4200001666F2D
:102B44000001636F000E00010001676F0001635113
:102B540036D0000100016751010DF350000100015E
:102B640065250001636FF450000100016621000136
:102B7400646F63C0F6FF64C0F7FF0800F5500009F6
:102B8400D8B422D0000100016751010DF3500001B7
:102B9400000165250001636FF45000010001662106
:102BA4000001646F63C0F6FF64C0F7FF0800000112
:102BB400F5CF62F01EEC10F000010001672B040E4B
:102BC400000100016765C5D7120000010001F3513F
:102BD400060DA40EF32400010001656F7E0EF4209F
:102BE4000001666F0001636F000E00010001676F52
:102BF4000001635136D0000100016751010DF3500B
:102C04000001000165250001636FF450000100011B
:102C140066210001646F63C0F6FF64C0F7FF08001B
:102C2400F5500009D8B422D0000100016751010D0C
:102C3400F3500001000165250001636FF4500001A9
:102C4400000166210001646F63C0F6FF64C0F7FFF2
:102C540008000001F5CF62F01EEC10F00001000145
:102C6400672B050E000100016765C5D7120000013E
:102C74000001EF51040D920EF32400010001656F71
:102C84007F0EF4200001666F0001636F000E0001E7
:102C94000001676F0001635136D0000100016751E4
:102CA400010DF3500001000165250001636FF4502C
:102CB4000001000166210001646F63C0F6FF64C077
:102CC400F7FF0800F5500009D8B422D00001000134
:102CD4006751010DF3500001000165250001636F88
:102CE400F4500001000166210001646F63C0F6FF27
:102CF40064C0F7FF08000001F5CF62F01EEC10F08D
:102D040000010001672B030E000100016765C5D7B0
:102D1400120000010001EC51050D790EF3240001AD
:102D24000001656F7F0EF4200001666F0001636F80
:102D3400000E00010001676F0001635136D00001ED
:102D440000016751010DF3500001000165250001E8
:102D5400636FF4500001000166210001646F63C0D9
:102D6400F6FF64C0F7FF0800F5500009D8B422D07C
:102D7400000100016751010DF350000100016525B8
:102D84000001636FF4500001000166210001646FCB
:102D940063C0F6FF64C0F7FF08000001F5CF62F0DE
:102DA4001EEC10F000010001672B040E000100016D
:102DB4006765C5D7120000010001F451060DEC0E41
:102DC400F32400010001656F7E0EF4200001666F9C
:102DD4000001636F000E00010001676F0001635181
:102DE40036D0000100016751010DF35000010001CC
:102DF40065250001636FF4500001000166210001A4
:102E0400646F63C0F6FF64C0F7FF0800F550000963
:102E1400D8B422D0000100016751010DF350000124
:102E2400000165250001636FF45000010001662173
:102E34000001646F63C0F6FF64C0F7FF080000017F
:102E4400F5CF62F01EEC10F000010001672B050EB7
:102E5400000100016765C5D7120000010001F151AE
:102E6400050DA60EF32400010001656F7F0EF4200A
:102E74000001666F0001636F000E00010001676FBF
:102E84000001635136D0000100016751010DF35078
:102E94000001000165250001636FF4500001000189
:102EA40066210001646F63C0F6FF64C0F7FF080089
:102EB400F5500009D8B422D0000100016751010D7A
:102EC400F3500001000165250001636FF450000117
:102ED400000166210001646F63C0F6FF64C0F7FF60
:102EE40008000001F5CF62F01EEC10F000010001B3
:102EF400672B040E000100016765C5D712000001AD
:102F04000001EB51040D280EF32400010001656F4C
:102F14007F0EF4200001666F0001636F000E000154
:102F24000001676F0001635136D000010001675151
:102F3400010DF3500001000165250001636FF45099
:102F44000001000166210001646F63C0F6FF64C0E4
:102F5400F7FF0800F5500009D8B422D000010001A1
:102F64006751010DF3500001000165250001636FF5
:102F7400F4500001000166210001646F63C0F6FF94
:102F840064C0F7FF08000001F5CF62F01EEC10F0FA
:102F940000010001672B030E000100016765C5D71E
:102FA400120008C563F01AEC0EF000010001666F10
:102FB4000001000166A10BD00001656F010E000144
:102FC4000001606F000165514CEC13F00AD0000160
:102FD400656F010E00010001606F000165518CEC0A
:102FE40013F00001000166A30BD00001656F020E0F
:102FF40000010001606F000165514CEC13F00AD030
:103004000001656F020E00010001606F000165514F
:103014008CEC13F00001000166A50BD00001656F74
:10302400030E00010001606F000165514CEC13F0C8
:103034000AD00001656F030E00010001606F0001FA
:1030440065518CEC13F01200000E486E000E496EB0
:103054004E50020AD8A41DD020EE01F03E50D926CD
:103064003F50DA22080EDF6E20EE02F03E50D926E1
:103074003F50DA22280EDE6E040EDD6E3EC0D9FF0C
:103084003FC0DAFF480EDF6E3EC0D9FF3FC0DAFF13
:103094002CD0000120EEFCF0040114EE26F0E652E0
:1030A400DE52DD50E55C02E1DF50E75CD8B004D0CD
:1030B40026C4FCF027C4FDF096EC1BF0000120EEC2
:1030C40002F00001DF51D9260001E051DA22280E76
:1030D400DE6E040EDD6EDFC0D9FFE0C0DAFF480EFD
:1030E400DF6EDFC0D9FFE0C0DAFF000EDB8E120016
:1030F40000010001F451D8A439D04DD0EBC061F0E7
:10310400010E0001626F0001612B03D00001D89011
:1031140062370001612FFAD700016251FF0A0001F2
:1031240000016017EBC061F0F2C062F00001612B96
:1031340003D00001D89062370001612FFAD710D074
:10314400EBC061F0FD0E00016127F2C062F00001E6
:10315400612B03D00001D89062370001612FFAD7A8
:103164000001625100010001601315D0000100014B
:10317400EB51000AD8B4C2D7010AD8B4BFD7030AA6
:10318400D8B4BCD7010AD8B4DBD7070AD8B4D8D787
:10319400010AD8B4D5D700010001605112007D0E98
:1031A40000010001666F950E0001656F0001616FFB
:1031B400000E00010001676F000161513FD0000162
:1031C40000016751010DF350000100016525000164
:1031D400616FF4500001000166210001626F61C05B
:1031E400F6FF62C0F7FF0800F55000010001601906
:1031F400D8A421D000010001F351070D950EF3244A
:103204000001616F7D0EF4200001626F0001000176
:103214006751010DF350000161250001636FF45003
:10322400000162210001646F63C0F6FF64C0F7FF10
:103234000800F5500BD000010001672B060E0001B9
:1032440000016765BCD700010001605112004B66A4
:103254005FD0010E4B6E4C665BD0010E4C6E4E502F
:10326400020AD8A418D0000120EE01F00001DF51B9
:10327400D9260001E051DA22000EDF6EDFC0D9FF4B
:10328400E0C0DAFF480EDF6EDFC0D9FFE0C0DAFF2E
:10329400000EDB8E3DD04E04D8A43AD0000E466E0C
:1032A40020EE01F03C50D9263D50DA22080EDF6EA4
:1032B40020EE02F03C50D9263D50DA22200EDE6E7C
:1032C400040EDD6E3CC0D9FF3DC0DAFF040EDF6E94
:1032D4003CC0D9FF3DC0DAFF000EDB8E010E466E06
:1032E40020EE01F03E50D9263F50DA22080EDF6E60
:1032F40020EE02F03E50D9263F50DA22200EDE6E38
:10330400040EDD6E3EC0D9FF3FC0DAFF800EDF6ED3
:103314001200000100016FC060F000010001616B48
:10332400000E00010001636F0C0E0001626F0DECD2
:103334001CF000010001605100010001746F53A0F2
:1033440049D0060E00010001746544D0070E000147
:103354000001745F000E00010001636F0C0E000198
:10336400626F000100016FC060F000010001616B39
:10337400F6EC1EF0000160C069F0000161C06AF063
:10338400000E000100016C6F050E00016B6FD1ECA3
:1033940010F0100E0001000169250001706F780E15
:1033A400000100016A210001716F000100017451E4
:1033B400010DF350000170250001726FF4500001FB
:1033C40071210001736F72C0F6FF73C0F7FF08002C
:1033D400F55001D0000E12000250D8B409D00150AB
:1033E400020D0001DF0EF324D96E0001000E08D097
:1033F4000150020D0001E30EF324D96E0001000E0A
:10340400F420DA6EDECF06F0DDCF07F007500610A9
:10341400D8A405D0000E026E000E016E40D020EE3E
:1034240002F00650D9260750DA2203C0DEFF04C09A
:10343400DDFF20EE01F00650D9260750DA2205C040
:10344400DFFF06C0D9FF07C0DAFF400EDF1606C053
:10345400D9FF07C0DAFF000EDB8606C0D9FF07C01C
:10346400DAFF000EDB8E0250D8B409D00150020DF1
:103474000001DF0EF324D96E0001000E08D00150C4
:10348400020D0001E30EF324D96E0001000EF420B6
:10349400DA6E040EDF1A06C001F007C002F0120053
:1034A4002D0E4D6E5C50FD0BD8A45CD05CC026F094
:1034B400D89026323F0E26162650040D0401000E25
:1034C400F3243C6E0401040EF4203D6E3CC03EF037
:1034D4003DC03FF0040E3E1A3CC0D9FF3DC0DAFFA8
:1034E400DF30E8320F0B0D0AD8A439D0266E000E57
:1034F400286E265024D020EE02F03C50D9263D50B0
:10350400DA22DECF26F0DDCF27F026C0D9FF27C090
:10351400DAFF2850010D0401200EF324E16E0401AA
:10352400040EF420E26EDFCFE7FF20EE02F03C5001
:10353400D9263D50DA22DE2A000EDD22282A070E83
:103544002864D9D720EE02F03C50D9263D50DA2227
:10355400200EDE6E040EDD6EF4EC14F009D049EC9E
:1035640010F006D05C50FD0B040AD8B424EC1BF018
:1035740012000101010E00010001616F0101840EBE
:103584000001606F000E00010001636F0E0E000168
:10359400626F000E00010001656F1E0E0001646F72
:1035A400C1EC0DF0000E00010001616F020E00017C
:1035B400606F9EEC0CF000010001F66F050E000137
:1035C4000001F66508D00001686F000E00010001DB
:1035D400F66F00016851000E00010001616F040ED6
:1035E4000001606F9EEC0CF000010001F36F050E0A
:1035F40000010001F36508D00001686F000E0001AE
:103604000001F36F00016851000E00010001616FB9
:10361400030E0001606F9EEC0CF000010001EF6FDF
:10362400040E00010001EF6508D00001686F000E70
:1036340000010001EF6F0001685171EC0DF05BECCB
:1036440014F01200DFC0D9FFE0C0DAFF0001DF3858
:10365400E832E832010B096E040E00010001DF1BA1
:1036640000010001EE51080AD8A40ED0040104019F
:1036740022517F0B6E6E6E50D8B402D0100E01D062
:10368400040E00010001EE6F4E04D8A42ED00001F8
:1036940020EE02F00001DF51D9260001E051DA22C8
:1036A400280EDE6E040EDD6E96EC1BF05650020AF8
:1036B400D8A406D0DFC0D9FFE0C0DAFF040E0DD0D5
:1036C400096606D0DFC0D9FFE0C0DAFF480E05D096
:1036D400DFC0D9FFE0C0DAFF080EDF6EDFC0D9FF1C
:1036E400E0C0DAFF000EDB8E1ED000010001DAAF6D
:1036F40018D000010001DE51DD11D8B40FD0000153
:1037040020EEDDF001D80AD00500FA6EDE50FD6E21
:10371400DE50FE6EF850FF6EFA50120000010001F8
:10372400DA9F000E4E6E1200016E080E026E0150FA
:10373400080E00010001FC5D000E0001FD59D8B027
:103744000BD0FCC002F0566602D0010E04D0560421
:10375400D8A402D0020E566E025000010001FC5F94
:10376400000E0001FD5B000120EE01F00001DF51BD
:10377400D9260001E051DA2202C0DFFF0401040E61
:10378400416E0401280E406E00010001FBA11FD010
:103794003FD00001F8C0F6FF0001F9C0F7FFF86A56
:1037A40040C0D9FF41C0DAFF070EF76403D0080018
:1037B400F55005D0F6CFE9FFF7CFEAFFEF50DF6E03
:1037C40000010001F84BF92B404A412A0206026627
:1037D400E0D720D00001F8C0F6FF0001F9C0F7FFE0
:1037E400F86A40C0D9FF41C0DAFF070EF76403D07E
:1037F4000800F55005D0F6CFE9FFF7CFEAFFEF5008
:10380400DF6E00010001F84BF92B404A412A020601
:103814000266E0D712000001646F000E000100018F
:10382400666F000164510001000161AF0FD0000117
:103834000001606D0001611FD8B0612B0001646F4D
:10384400010E00010001666F0001645100010001D6
:1038540063AF07D000010001626D0001631FD8B09F
:10386400632B0001000163516211D8B43AD0000106
:10387400646F010E00010001656F0001645109D0FD
:10388400000100010001D890623763370001000194
:10389400652B0001000163AFF3D700010001625101
:1038A40000010001605D000100016351000100019D
:1038B4006159D8A00CD0000100016251000100013F
:1038C400605F00010001635100010001615B0001C0
:1038D40000010001D8906333623300010001652FB9
:1038E400DCD7000100016651D8B407D00001000103
:1038F400606D0001611FD8B0612B60C060F061C0D1
:1039040061F01200000E04010401286F000E04018E
:103914000401296F4DD000010001FB8F000100015B
:10392400ED05D8A452D00401040128834ED000012F
:103934000001FB8F4AD000010001FB8F0401040148
:1039440024BF0ED00401040124510F0B016E015059
:10395400020D0001E30EF324D96E0001000E0DD018
:103964000401040124510F0B016E0150020D0001EA
:10397400DF0EF324D96E0001000EF420DA6EDECFE0
:1039840002F0DDCF03F002C0D9FF03C0DAFFDF503D
:10399400016E01AE1AD002C0D9FF03C0DAFFDF50B6
:1039A400016E01A412D0010E04010401286F0DD090
:1039B4000401040120511F0B000AD8B4ACD7010A3A
:1039C400D8B4B5D7030AD8B4B6D700010001FBAF09
:1039D40010D00401040E00010001F96F0401280E47
:1039E4000001F86F00010001FB81020E00010001DB
:1039F400FC6F12006D9800010001FBBF3AD000017A
:103A04000001DAAF0BD0020E4E6E496602D026ECEE
:103A140018F0000E4C6E000E4B6E66D020EE01F0D6
:103A24003E50D9263F50DA22080EDF6E20EE02F017
:103A34003E50D9263F50DA22200EDE6E040EDD6E93
:103A44003EC0D9FF3FC0DAFF0C0EDF6E3EC0D9FF87
:103A54003FC0DAFF000EDB8EDFC0D9FFE0C0DAFF23
:103A6400040EDF6EDFC0D9FFE0C0DAFF000EDB8E8C
:103A74003BD00401040120AF0FD0010E4E6E486606
:103A840002D026EC18F0000E4C6E000E4B6E4A6607
:103A94002BD029EC19F028D0020E4E6E20EE01F046
:103AA4003E50D9263F50DA22080EDF6E20EE02F097
:103AB4003E50D9263F50DA22200EDE6E040EDD6E13
:103AC4003EC0D9FF3FC0DAFF040EDF6E3EC0D9FF0F
:103AD4003FC0DAFF000EDB8E000E4C6E000E4B6E04
:103AE4004A6602D029EC19F0120000010001FB8F94
:103AF4000F0E026E710E016E000E046E000E036E48
:103B0400000E066E010E056EFFEC0CF00401040EAF
:103B1400026E0401000E016E000E046E000E036EB0
:103B2400000E066E200E056EFFEC0CF06D8C1C6E04
:103B3400000E1D6E1C5019D01D50010D0001E70E22
:103B4400F324D96E0001000EF420DA6E000EDF6E4D
:103B54001D50010D0001E90EF324D96E0001000E81
:103B6400F420DA6E000EDF6E1D2A010E1D64E4D708
:103B7400000E026E5B0E016E000E046E000E036EEC
:103B8400000E066E010E056EFFEC0CF06D9C040138
:103B9400040E00010001E06F0401080E0001DF6F54
:103BA4000401040E3D6E0401000E3C6E3CC03EF068
:103BB4003DC03FF022C45AF05A6602D0100E0FD016
:103BC400000E156E010E146E000E176E5A0E166E50
:103BD400000E196E010E186E6CEC12F0200E00012E
:103BE4000001EE6F1200000100016151D8B40BD046
:103BF400000100016051020D0001DF0EF324D96EB3
:103C04000001000E0AD0000100016051020D000104
:103C1400E30EF324D96E0001000EF420DA6E0001E5
:103C2400DECF65F00001DDCF66F0000100016651D2
:103C34006511D8A408D0000E00010001616F000EC8
:103C44000001606F4FD0000120EE02F000016551C9
:103C5400D92600016651DA22000162C0DEFF0001AC
:103C640063C0DDFF000120EE01F000016551D9269B
:103C740000016651DA22000164C0DFFF65C0D9FF8C
:103C840066C0DAFF400EDF1665C0D9FF66C0DAFFF2
:103C9400000EDB8665C0D9FF66C0DAFF000EDB8E3E
:103CA400000100016151D8B40BD000010001605142
:103CB400020D0001DF0EF324D96E0001000E0AD0BC
:103CC400000100016051020D0001E30EF324D96EDE
:103CD4000001000EF420DA6E040EDF1A65C060F0F5
:103CE40066C061F01200040104012039E832030BBC
:103CF4000009D8A478D055D000010001FB8F080E2C
:103D040000010001EE6F6FD023EC23F06CD077EC50
:103D14001DF069D0000E00010001F96F5A0E000178
:103D2400F86F14D084EC1CF05ED050EC28F05BD01B
:103D3400040104012451010D5B0EF324246E000ED2
:103D4400F420256E24C0F8F025C0F9F0000100012C
:103D5400FB81010E00010001FC6F00010001FB8FDB
:103D640042D000010001FB8F040104012451010D24
:103D74005B0EF324D96E000EF420DA6E040122C423
:103D8400DFFF31D0000E156E020E146E000E176E9A
:103D9400000E166E000E196E000E186E6CEC12F00A
:103DA40022D0040104012151000AD8B4BBD7010A6E
:103DB400D8B4BBD7020AD8B4B8D7060AD8B49CD7AB
:103DC400030AD8B4A1D7010AD8B4DCD70F0AD8B4EF
:103DD400A1D7010AD8B49BD7030AD8B4A9D7010A3A
:103DE400D8B4BFD7070A12000001646F000E0001A7
:103DF4000001666F000164510001000163AF0FD040
:103E040000010001626D0001631FD8B0632B000143
:103E1400646F010E00010001666F0001645100012E
:103E2400000161AF0BD000010001606D0001611F52
:103E3400D8B0612B010E00010001661B000E0001C9
:103E44000001686F000E0001676F000100016351FB
:103E54006211D8B443D00001646F010E0001000167
:103E6400656F0001645109D0000100010001D89080
:103E74006237633700010001652B0001000163AF65
:103E8400F3D7000100010001D890673768370001BB
:103E94000001625100010001605D000100016351F5
:103EA400000100016159D8A00FD000010001625146
:103EB40000010001605F0001000163510001000185
:103EC400615B000100016781000100010001D890DD
:103ED4006333623300010001652FD3D70001000171
:103EE4006651D8B407D000010001676D0001681F56
:103EF400D8B0682B67C060F068C061F0120062C07F
:103F04006AF063C06BF060C068F061C069F00001E2
:103F140000016851000100016A5D0001000169515E
:103F2400000100016B59D8B053D000016AC066F09B
:103F340000016BC067F000010001645100016627B5
:103F44000001000165510001672300016651000171
:103F54000001685D00016751000100016959D8B092
:103F640037D0000100016451000100016A270001FB
:103F740000016551000100016B230001000164513F
:103F840000010001682700010001655100010001E2
:103F94006923000100016A07D8A06B076AC0D9FF32
:103FA4006BC0DAFF000100016807D8A0690768C088
:103FB400E1FF69C0E2FFDFCFE7FF00010001640712
:103FC400D8A06507000165516411D8B423D0E1D7A6
:103FD4000001000165516411D8B41CD06AC0D9FF36
:103FE4006BC0DAFF68C0E1FF69C0E2FFDFCFE7FF23
:103FF400000100016A4B6B2B00010001684B692B27
:10400400000100016407D8A065070001655164112F
:10401400D8A4E4D7120000010001F651020AD8B472
:1040240006D000010001F651030AD8A42BD04F0E8C
:10403400000100016F6526D0540E000100016F617C
:1040440021D0B00E000100016F2500010001696F4D
:10405400000100016A6BFF0E6A23000E00010001DB
:104064006C6F030E00016B6FD1EC10F0CC0E0001ED
:1040740000016925000100016F6F7F0E000100013E
:104084006A2157D0000E00010001636F0C0E00017D
:10409400626F000100016FC060F000010001616BFC
:1040A400F6EC1EF0000160C069F0000161C06AF026
:1040B400000E000100016C6F240E00016B6FD1EC47
:1040C40010F04B0E0001000169250001716F780E9C
:1040D400000100016A210001726F000E000100015D
:1040E400636F0C0E0001626F000100016FC060F08D
:1040F40000010001616B0DEC1CF0000160C069F06F
:10410400000161C06AF0000E000100016C6F030E33
:1041140000016B6FD1EC10F0000100016951000146
:104124007125000100016F6F000100016A51000157
:1041340072210001706F12000401040120511F0B51
:10414400016E0104D8A48CD0040104012451D8A424
:1041540087D0040104012151060AD8B424D02DD0FB
:104164005A04D8A42AD07D0E00010001F96FFB0E79
:104174000001F86F000E00010001FD6F090E0CD064
:104184007C0E00010001F96FF50E0001F86F000EBE
:1041940000010001FD6F400E0001FC6FC00E000124
:1041A4000001FB6F0AD0040104012351210AD8B491
:1041B400D7D7030AD8B4E4D7010A0401040120398B
:1041C400E832030B016E0104D8A44AD034D08BEC3E
:1041D4000DF046D0000E00010001F96F5E0E0001E3
:1041E400F86F000E00010001FD6F010E0001FC6F6D
:1041F400C10E16D0800E00010001FB6F23C45EF0D7
:104204002FD0000E00010001F96F5D0E0001F86F60
:10421400000E00010001FD6F010E0001FC6F810E14
:1042240000010001FB6F1CD0800E00010001FB6F38
:1042340022C45DF015D0040104012151010AD8B44F
:104244000FD0030AD8B4C6D7010AD8B4DAD70A0AF9
:10425400D8B4BDD7030AD8B4CDD7010AD8B4E4D7AB
:104264001200FE0EF66E170EF76E0900F5CF7DF004
:104274000900F5CF7EF0020E00017D5D000E7E592F
:10428400D8A023D0000100017B510C0DD00EF324E3
:1042940000017D6F750EF42000017E6F00010001A6
:1042A4007C51010DF35000017D2500017F6FF45016
:1042B40000017E210001806F7FC0F6FF80C0F7FF00
:1042C40008000001F5CF81F00BD0000100017B5103
:1042D4000C0DF350000100017C2500010001816FE9
:1042E400000100017C51010D0101A20EF324D96EDD
:1042F4000101010EF420DA6EDF2A000100017B5176
:10430400010D0101B60EF324D96E0101010EF42052
:10431400DA6EDF2A81C075F0CFEC29F000010001CC
:10432400826FDF0E0001000182651AD0E80E0001E1
:104334000001826115D082C07DF0200E00017D272E
:10434400010E00017E6F00017D2B03D00001D89087
:104354007E3700017D2FFAD700017E51541223D0FD
:10436400000100018251F00AD8A404D00101010126
:10437400AF8119D000010001FF51800A780FD8B035
:1043840012D000010001FF51010D0101AE0EF32412
:10439400D96E0101010EF420DA6E000181C0DFFF45
:1043A40000010001FF2B120020EE01F03C50D92641
:1043B4003D50DA22DF500B6E0B5000010001DB5D33
:1043C400000E0001DC59D8A0DBC00BF00B5000013B
:1043D4000001DB5F000E0001DC5B096E000E0A6E5B
:1043E400095015D00A50010D0401280EF324D96E8A
:1043F4000401040EF420DA6ED7C0E1FFD8C0E2FF56
:10440400DFCFE7FF00010001D74BD82B0A2A0B505E
:104414000A5CD8A0E7D700010001DC51DB11D8B455
:104424002DD020EE01F03E50D9263F50DA22080E5E
:10443400DF6E20EE02F03E50D9263F50DA22280EDD
:10444400DE6E040EDD6E3CC0D9FF3DC0DAFFDF50E6
:10445400096E09BC06D03EC0D9FF3FC0DAFF480E42
:1044640005D03EC0D9FF3FC0DAFF080EDF6E3EC064
:10447400D9FF3FC0DAFF000EDB8E3AD020EE01F008
:104484003E50D9263F50DA22080EDF6E20EE02F0AD
:104494003E50D9263F50DA22200EDE6E040EDD6E29
:1044A4003EC0D9FF3FC0DAFF040EDF6E3EC0D9FF25
:1044B4003FC0DAFF000EDB8E00010001DE51DD118A
:1044C400D8B40FD0000120EEDDF001D80AD00500E9
:1044D400FA6EDE50FD6EDE50FE6EF850FF6EFA503E
:1044E400120000010001DA9F4A6602D029EC19F09B
:1044F40012000001686F000E000100016A6F0001E4
:1045040068510001686F000E000100016B6F00012B
:1045140068510001686F000E000100016D6F000119
:10452400685115D0000100016D51010D0101B60E55
:10453400F324D96E0101010EF420DA6E010EDF645A
:1045440003D0000100016A2B000100016D2B070E4E
:10455400000100016D65E6D70001686F000E0001DF
:1045640000016D6F0001685115D0000100016D510B
:10457400010D0101A20EF324D96E0101010EF420F4
:10458400DA6E010EDF6403D0000100016B2B000121
:1045940000016D2B0B0E000100016D65E6D70001D3
:1045A400686F000E000100016C6F00016851010E7C
:1045B400000100016A650DD0010E000100016B6568
:1045C40008D00001686F010E000100016C6F00014A
:1045D40068516CC069F00101010E00010001616FB6
:1045E4000101B60E0001606F000E00010001636F4F
:1045F400000E0001626F000E00010001656F080EDD
:104604000001646FC1EC0DF00101010E0001000115
:10461400616F0101A20E0001606F000E0001000134
:10462400636F000E0001626F000E00010001656FF0
:104634000C0E0001646FC1EC0DF000010001695122
:104644001200040104012051800AD8A4A4D0C00E91
:1046540000010001FB6F92D07F0E00010001F96F91
:10466400BA0E0001F86F000E00010001FD6F120E7A
:104674000001FC6F90D00401040122677AD0040188
:1046840004012251020D490EF324F66E780EF42033
:10469400F76E09000001F5CFF8F00A000001F5CF2C
:1046A400F9F0020E00010001F825016E000E000170
:1046B4000001F921026E0150F66EE96E070EEA6EF2
:1046C4000250EA6403D0EA6EEF5003D0F76E08009C
:1046D400F55000010001FC6F030E00010001F825F4
:1046E400016E000E00010001F921026E0150F66E08
:1046F400E96E070EEA6E0250EA6403D0EA6EEF50E8
:1047040003D0F76E0800F55000010001FD6F43D09F
:10471400030E0401040122612CD00401040122517E
:10472400020D3F0EF324F66E780EF420F76E0900A6
:104734000001F5CFF8F00A000001F5CFF9F000010F
:104744000001F851F66EE96E070EEA6E00010001F1
:10475400F951EA6403D0EA6EEF5003D0F76E080013
:10476400F550016E015000010001FC6F0001FD6B6A
:1047740012D0000E00010001FB6F0DD004010401F2
:104784002351010AD8B468D7030AD8B474D7010AEC
:10479400D8B4BED7EED7120000010001EE05D8B49C
:1047A4006DBA08D0000E686E69806988020E000137
:1047B4000001EE6F68B469A403D068942BEC0DF08B
:1047C4006DB297D068B069A008D02EEC25F0A08A0D
:1047D400040E00010001EE6F689068B869A803D068
:1047E400EBEC0CF0689868AC18D069AC0ED0000EF5
:1047F400156E730E146E000E176E000E166E000EFC
:10480400196E010E186E6CEC12F0689C4D50D8A411
:104814004D064D6602D029EC19F068BA69AA02D097
:10482400FBEC0DF068B269A210D07F0E156EFF0E7E
:10483400146E000E176E000E166E000E196E010E29
:10484400186E6CEC12F0000E6A6E040E000100018A
:10485400EE6101D04ED069A64CD0296E000E2B6EAD
:10486400295044D068A645D06CCF5CF05C30E83267
:10487400E8320F0B506E68965CB40BD0010E296EB3
:104884005050010D0001E90EF324D96E0001000E11
:104894000AD0010E296E5050010D0001E70EF324D9
:1048A400D96E0001000EF420DA6E0001DF50010B16
:1048B4002A6E29502A1A0001DF502A18FE0B2A18E2
:1048C4000001DF6E506603D052EC1AF00ED0000ED9
:1048D400156E720E146E000E176E5C0E166E000EC0
:1048E400196E000E186E6CEC12F02B2A030E2B645A
:1048F400B9D7A19A12009FD0A7C084F0A8C085F0B0
:10490400A9C086F0AAC087F0ABC088F0ACC089F01B
:104914007B0E000100018B6FB70E00018A6F7C0EC5
:10492400000100018D6F0B0E00018C6F7C0E0001E5
:1049340000018F6F5F0E00018E6F06EC36F08BD096
:10494400A7C084F0A8C085F0A9C086F0AAC087F0EB
:10495400ABC088F0ACC089F07A0E000100018B6F07
:10496400130E00018A6F7A0E000100018D6F670E2D
:1049740000018C6F7A0E000100018F6FBB0E0001E5
:104984008E6F06EC36F067D0A7C084F0A8C085F01F
:10499400A9C086F0AAC087F0ABC088F0ACC089F08B
:1049A400790E000100018B6F6B0E00018A6F790E86
:1049B400000100018D6FBF0E00018C6F790E0001A4
:1049C40000018F6FBF0E00018E6F06EC36F043D0EE
:1049D400A7C084F0A8C085F0A9C086F0AAC087F05B
:1049E400ABC088F0ACC089F07B0E000100018B6F76
:1049F4000F0E00018A6F7B0E000100018D6F630EA4
:104A040000018C6F7B0E000100018F6F630E0001AB
:104A14008E6F06EC36F01FD0A7C07BF0A8C07CF0E8
:104A2400A9C07DF0AAC07EF0ABC07FF0ACC080F01E
:104A3400A4EC26F010D000010001F451010AD8B40E
:104A44007FD7030AD8B4A0D7010AD8B455D7070A28
:104A5400D8B4BED7E1D71200A09A000E6A6E000E39
:104A6400686E000E706E0F0E026E710E016E000EF7
:104A7400046E000E036E000E066E010E056EFFEC52
:104A84000CF0160E6F6E9F0E6B6E7B0E696E096EC8
:104A9400000E0A6E095015D00A50040D0401000ED0
:104AA400F324D96E0401040EF420DA6E000EDE6ED7
:104AB400000EDE6E000EDE6E000EDD6EDD52DD5287
:104AC4000A2A070E0A64E8D76D8C000E6E6E6D9884
:104AD4006D9C10D06896000E00010001FB6F000E63
:104AE40000010001DA6F000E00010001DC6F000E0E
:104AF4000001DB6F68B6EED7010E4B6E010E4C6EF3
:104B0400000E486E000E496E000E476E096E000ED0
:104B14000A6E095035D00A50020D0001DF0EF3244D
:104B2400D96E0001000EF420DA6E000EDE6E000E67
:104B3400DD6E0A50020D0001E30EF324D96E00016C
:104B4400000EF420DA6E000EDE6E000EDD6E0A50EA
:104B5400010D0001E70EF324D96E0001000EF420CC
:104B6400DA6E000EDF6E0A50010D0001E90EF32427
:104B7400D96E0001000EF420DA6E000EDF6E0A2AF0
:104B8400010E0A64C8D70401040E00010001E06F9D
:104B94000401080E0001DF6F160E706E040E04018E
:104BA4000401036F200E0401026F080E04010401C6
:104BB400016F040E04010401006F04010401008F5D
:104BC400000E5A6E000E00010001EE6F12007F0EFF
:104BD40000010001646F440E0001636F76EC10F075
:104BE400FE0EF66E170EF76E09000001F5CF60F0A9
:104BF4000A000001F5CF61F0DDEC0DF000010001C9
:104C0400626F1EEC10F00001696F280E00010001B4
:104C1400626F000169511EEC10F07F0E000100016B
:104C2400646FD80E0001636F76EC10F0000E000183
:104C34000001616F000E0001606FDDEC0DF00001FA
:104C44000001626F1EEC10F00001696F370E000165
:104C54000001626F000169511EEC10F0000E0001AA
:104C64000001616F010E0001606FDDEC0DF00001C9
:104C74000001626F1EEC10F0000E00010001616F74
:104C8400000E0001606FDDEC0DF000010001626FA9
:104C94001EEC10F00001696F280E00010001626F24
:104CA400000169511EEC10F07E0E00010001646FDA
:104CB400120E0001636F76EC10F095EC15F07F0E88
:104CC40000010001646FDE0E0001636F76EC10F0EA
:104CD4008BEC16F07F0E00010001646FE20E000100
:104CE400636F76EC10F0DDEC16F07F0E000100012E
:104CF400646FE60E0001636F76EC10F039EC16F089
:104D04007F0E00010001646FEA0E0001636F76EC10
:104D140010F0E7EC15F07F0E00010001646FEE0E59
:104D24000001636F76EC10F02FEC17F07F0E00019A
:104D34000001646FF20E0001636F76EC10F081ECF9
:104D440017F012000001816F020E00010001846F50
:104D5400000181517BC0D9FF7CC0DAFFDF50000124
:104D64000001826F0001816F020E00010001856F56
:104D740000018151A7D0000100018551010DF350BC
:104D8400000100017B25D96EF450000100017C2153
:104D9400DA6EDF5000010001836F83C06FF08BEC8B
:104DA40019F000010001866F00010001866707D039
:104DB40083C075F0CFEC29F000010001866F00017B
:104DC40000018651D8B47BD0080E00010001846133
:104DD40076D0000100018651900AD8A404D00001C5
:104DE400816F010E09D0000100018651910AD8A4F7
:104DF40007D00001816F000E00010001F26F49D05D
:104E0400000100018651390AD8A42CD0020E0001F9
:104E140000017D2500010001606F000E000100010A
:104E24007E210001616F0001000186C062F0000173
:104E34000001636B000E00010001656F060E0001A6
:104E4400646FDAEC12F0000100016151000160119D
:104E5400D8A421D01AEC0FF00009D8B41CD0010E4C
:104E64004F1A19D0000100018651270AD8A413D083
:104E7400000100018251220BD8B40DD01AEC0FF0BE
:104E84000009D8B408D00001816F870E0001000129
:104E9400866F00018151000100018451010DF3501E
:104EA400000100017F25D96EF4500001000180212A
:104EB400DA6E000186C0DFFF00010001842B0001CF
:104EC4000001852B070E00010001856554D77FC0C2
:104ED400D9FF80C0DAFF000182C0DFFF010E12009B
:104EE400A09A000E6A6E000E686E000E706E0F0EB1
:104EF40000010001616F710E0001606F000E00017E
:104F04000001636F000E0001626F000E00010001DA
:104F1400656F010E0001646FC1EC0DF0160E6F6E2B
:104F24009F0E6B6E7B0E696E0001686F000E0001B0
:104F34000001696F0001685119D000010001695135
:104F4400040D0401000EF324D96E0401040EF420B0
:104F5400DA6E000EDE6E000EDE6E000EDE6E000EE9
:104F6400DD6EDD52DD5200010001692B070E0001E8
:104F740000016965E2D76D8C000E6E6E6D986D9CB4
:104F840010D06896000E00010001FB6F000E0001B6
:104F94000001DA6F000E00010001DC6F000E000159
:104FA400DB6F68B6EED7010E4B6E010E4C6E000E31
:104FB400486E000E496E000E476E0001686F000EC9
:104FC40000010001696F000168513FD00001000138
:104FD4006951020D0001DF0EF324D96E0001000EA9
:104FE400F420DA6E000EDE6E000EDD6E00010001AC
:104FF4006951020D0001E30EF324D96E0001000E85
:10500400F420DA6E000EDE6E000EDD6E000100018B
:105014006951010D0001E70EF324D96E0001000E61
:10502400F420DA6E000EDF6E000100016951010DFB
:105034000001E90EF324D96E0001000EF420DA6EAB
:10504400000EDF6E00010001692B010E000100015A
:105054006965BCD70401040E00010001E06F04017E
:10506400080E0001DF6F160E706E040E04010401B9
:10507400036F200E0401026F080E04010401016F86
:10508400040E04010401006F04010401008F000EEA
:105094005A6E000E00010001EE6F120004010401BB
:1050A4002205D8A416D00401040120511F0B0009C5
:1050B400D8A40FD000010001FB8F04010401215189
:1050C400030AD8A402D0010E01D0000E0001000191
:1050D400ED6F0401040122675FD104010401205132
:1050E4001F0B020AD8A458D10401040124510F0B48
:1050F4000009D8B451D10401040124510F0B1C6ED2
:10510400020E1C5CD8B048D100010001EE51200A07
:10511400D8A442D100010001FB8F0401040124BF83
:1051240021D00401040124510F0B1C6E1C50020DEC
:105134000001E30EF324D96E0001000EF420DA6EB0
:10514400DECF22F0DDCF23F00401040124510F0B44
:105154001C6E1C50010D0001E90EF324D96E0001F0
:10516400000E20D00401040124510F0B1C6E1C50AE
:10517400020D0001DF0EF324D96E0001000EF420AD
:10518400DA6EDECF22F0DDCF23F0040104012451D6
:105194000F0B1C6E1C50010D0001E70EF324D96E99
:1051A4000001000EF420DA6EDF50216E21B002D02F
:1051B400229401D022840401040124BF0ED00401EE
:1051C400040124510F0B1C6E1C50020D0001E30E50
:1051D400F324D96E0001000E0DD004010401245102
:1051E4000F0B1C6E1C50020D0001DF0EF324D96E50
:1051F4000001000EF420DA6E22C0DEFF23C0DDFFC2
:10520400040104012151030AD8A439D022C0D9FFD2
:1052140023C0DAFFDF501C6E1CAE24D0040104014D
:1052240024BF0ED00401040124510F0B1C6E1C502A
:10523400010D0001E90EF324D96E0001000E0DD01A
:105244000401040124510F0B1C6E1C50010D0001BC
:10525400E70EF324D96E0001000EF420DA6E020E7C
:105264000001DF1222C0D9FF23C0DAFF000EDB8465
:1052740022C0D9FF23C0DAFF000EDB8E8DD0040ECE
:10528400221A22C0D9FF23C0DAFFDF501C6E1CAEE5
:105294001BD022C0D9FF23C0DAFF7F0EDF1622C045
:1052A400D9FF23C0DAFF000EDB8C000E156E050E4D
:1052B400146E22C016F023C017F0000E196E020EF1
:1052C400186E6CEC12F006D022C0D9FF23C0DAFFAE
:1052D400000EDB8C040E221A21B208D022C0D9FFA2
:1052E40023C0DAFFDF501C6E1CAE39D00401040168
:1052F40024BF0ED00401040124510F0B1C6E1C505A
:10530400010D0001E90EF324D96E0001000E0DD049
:105314000401040124510F0B1C6E1C50010D0001EB
:10532400E70EF324D96E0001000EF420DA6EFD0EB0
:105334000001DF1622C0D9FF23C0DAFF3B0EDF16BF
:10534400000E156E050E146E22C016F023C017F061
:10535400000E196E020E186E6CEC12F006D022C00C
:10536400D9FF23C0DAFF3B0EDF16040104012451E8
:105374000F0B1C6E1C50010D700EF3241D6E0F0ECE
:10538400F4201E6E1DC01FF01EC020F01FC0D9FFE8
:1053940020C0DAFFFE0EDF16120075C06FF08BEC32
:1053A40019F0000100017A6F000100017A51D8B4AC
:1053B40082D1000100017A5195D1000E0001000153
:1053C400636F0C0E0001626F0001000175C060F094
:1053D40000010001616BF6EC1EF0000160C069F091
:1053E400000161C06AF0000E000100016C6F0C0E38
:1053F40000016B6FD1EC10F0B00E000100016925C3
:105404000001766F770E000100016A210001776FB9
:105414000001000175C060F000010001616B000E25
:1054240000010001636F0C0E0001626F0DEC1CF0B3
:105434002BD1000E00010001636F0C0E0001626F9E
:105444000001000175C060F000010001616BF6EC21
:105454001EF0000160C069F0000161C06AF0000E36
:10546400000100016C6F0C0E00016B6FD1EC10F0A9
:10547400900E0001000169250001766F760E00018F
:1054840000016A210001776F0001000175C060F01E
:1054940000010001616B000E00010001636F0C0E3E
:1054A4000001626F0DEC1CF0EFD0000E0001000152
:1054B400636F0C0E0001626F0001000175C060F0A3
:1054C40000010001616BF6EC1EF0000160C069F0A0
:1054D400000161C06AF0000E000100016C6F0C0E47
:1054E40000016B6FD1EC10F0300E00010001692552
:1054F4000001766F760E000100016A210001776FCA
:105504000001000175C060F000010001616B000E34
:1055140000010001636F0C0E0001626F0DEC1CF0C2
:10552400B3D0000E00010001636F0C0E0001626F26
:105534000001000175C060F000010001616BF6EC30
:105544001EF0000160C069F0000161C06AF0000E45
:10555400000100016C6F0C0E00016B6FD1EC10F0B8
:10556400F00E0001000169250001766F760E00013E
:1055740000016A210001776F0001000175C060F02D
:1055840000010001616B000E00010001636F0C0E4D
:105594000001626F0DEC1CF077D0000E00010001D9
:1055A400636F0C0E0001626F0001000175C060F0B2
:1055B40000010001616BF6EC1EF0000160C069F0AF
:1055C400000161C06AF0000E000100016C6F0C0E56
:1055D40000016B6FD1EC10F0500E00010001692541
:1055E4000001766F770E000100016A210001776FD8
:1055F4000001000175C060F000010001616B000E44
:1056040000010001636F0C0E0001626F0DEC1CF0D1
:105614003BD0000E00010001636F0C0E0001626FAD
:105624000001000175C060F000010001616BF6EC3F
:105634001EF0000160C069F0000161C06AF0000E54
:10564400000100016C6F0C0E00016B6FD1EC10F0C7
:10565400B00E0001000169250001766F770E00018C
:1056640000016A210001776F0001000175C060F03C
:1056740000010001616B000E00010001636F0C0E5C
:105684000001626F0DEC1CF000010001605100018B
:1056940076250001786F0001000161510001772136
:1056A4000001796F78C0F6FF79C0F7FF08000001A8
:1056B400F5CF7AF013D000010001EC51000AD8B400
:1056C4007CD6010AD8B4B5D6030AD8B4EED6010AFA
:1056D400D8B427D7070AD8B460D79BD77AC060F06C
:1056E400D1EC18F0120000016E6F020E00010001EF
:1056F400726F00016E519ED1000100017251010DC3
:10570400F350000100016C25D96EF4500001000132
:105714006D21DA6E680E0FD0000100017251010D87
:10572400F350000100016C25D96EF4500001000112
:105734006D21DA6E690EDF6E7AD1000100017251BB
:10574400010DF350000100016C25D96EF4500001E5
:1057540000016D21DA6EDF508A0AD8B40AD0010A3A
:10576400D8B407D01B0AD8B4C7D7010AD8B4D4D741
:105774005ED1000100017251010DF35000010001DE
:105784006C25D96EF450000100016D21DA6E2C0EE7
:10579400D2D700010001F351020AD8B406D00001A7
:1057A4000001F351050AD8A442D16CC0D9FF6DC0E1
:1057B400DAFF000EDB84000100017251010DF35089
:1057C400000100016C2500010001606FF45000012C
:1057D40000016D210001616F000100017251010D92
:1057E400F350000100016C2500016E6FF4500001BC
:1057F40000016D2100016F6F010E00016E27000E84
:105804006F236EC062F06FC063F00001000172513B
:105814000001706F716B0001701F711F704B712B51
:10582400070E0001702500010001646F000E0001E5
:1058340071210001656F81EC1FF0000120EE07F07B
:1058440000016C51D92600016D51DA22000EDF6E81
:10585400000100017207EBD0000100017251010D3B
:10586400F350000100016C25D96EF45000010001D1
:105874006D21DA6EDF50650AD8B48BD7EF0AD8B43D
:1058840078D7010AD8B475D7D2D00001000172517B
:10589400010DF350000100016C25D96EF450000194
:1058A40000016D21DA6E8A0E0FD0000100017251E1
:1058B400010DF350000100016C25D96EF450000174
:1058C40000016D21DA6E8B0EDF6E6CC0D9FF6DC0E6
:1058D400DAFF030EDF12ABD0000100017251010D9B
:1058E400F350000100016C25D96EF4500001000151
:1058F4006D21DA6EDF50900AD8B4C7D7010AD8B444
:10590400D4D795D0000100017251010DF35000016C
:1059140000016C25D96EF450000100016D21DA6E8E
:10592400350E09D7000100017251010DF350000139
:1059340000016C25D96EF450000100016D21DA6E6E
:10594400DF50900AD8B4DED7010AD8B4DBD76FD0C1
:10595400000100017251010DF350000100016C259A
:10596400D96EF450000100016D21DA6E2C0EDF6E49
:105974006CC0D9FF6DC0DAFF000EDB8458D0000183
:1059840000017251010DF350000100016C25D96E24
:10599400F450000100016D21DA6EDF50900AD8B492
:1059A400D7D7010AD8B4D4D742D00001000172512C
:1059B400010DF350000100016C25D96EF450000173
:1059C40000016D21DA6E2C0EDF6E6CC0D9FF6DC044
:1059D400DAFF000EDB822BD0000100017251010DB1
:1059E400F350000100016C25D96EF4500001000150
:1059F4006D21DA6EDF50900AD8B4D7D7010AD8B433
:105A0400D4D715D000010001F651000AD8B495D6B8
:105A1400010AD8B421D7030AD8B45ED7010AD8B48E
:105A240081D7070AD8B4ABD7010AD8B4D5D70001B7
:105A34000001722B070E000100017265E3D712000A
:105A44000001C16F000E00010001C56F0001C151CA
:105A54007BEC22F00009D8B412D098D100010001E7
:105A6400FF51010D0101AE0EF324D96E0101010EA7
:105A7400F420DA6E0E0EDF6E00010001FF2B000130
:105A84000001FF51800A780FD8A0E8D70001000177
:105A9400F051060D0101840EF32400010001606F32
:105AA4000101010EF4200001616FB00E0001C16F0D
:105AB400010EC26FC1C062F0C2C063F0000E0001EB
:105AC4000001656F060E0001646F81EC1FF054C085
:105AD400AEF100010001EF51000800010001F025C2
:105AE400050F00010001C76F040E00010001C76526
:105AF40004D0050E00010001C75F00010001C75179
:105B0400040F00010001C96F040E00010001C96502
:105B140004D0050E00010001C95F0001C16F020E2F
:105B240000010001FF6F0001C1510001C16F000EAF
:105B340000010001C86F0001C1515CD000010001E7
:105B4400C751060D0101840EF3240001C16F010148
:105B5400010EF4200001C26F00010001C851010DC3
:105B6400F3500001C125D96EF4500001C221DA6E50
:105B7400DF5000010001C66F00010001C951060D8C
:105B84000101840EF3240001C16F0101010EF42010
:105B94000001C26FC1C060F0C2C061F00001000129
:105BA400C6C062F000010001636B000E0001000139
:105BB400656F060E0001646FDAEC12F0000100015B
:105BC400615100016011D8B412D000010001FF51ED
:105BD400010D0101AE0EF324D96E0101010EF42072
:105BE400DA6E0001C6C0DFFF00010001FF2B0001D7
:105BF4000001C82B050E00010001C8659FD711D014
:105C040000010001FF51010D0101AE0EF324D96E14
:105C14000101010EF420DA6E0E0EDF6E00010001A8
:105C2400FF2B00010001FF51800A780FD8A0E8D7AC
:105C340053A403D001010101AF810101010E000150
:105C44000001616F0101AE0E0001606F0101010EE0
:105C540000010001636F0101C90E0001626F000EB3
:105C640000010001656F080E0001646FA7EC14F0D9
:105C740000010001615100016011D8B480D0B00E60
:105C84000001C16F010EC26FC1C060F0C2C061F0FB
:105C9400CB0E0001C36F010EC46FC3C062F0C4C059
:105CA40063F0000E00010001656F060E0001646FD1
:105CB400A7EC14F000010001615100016011D8A4A7
:105CC40010D001010101B0510E0AD8B40AD001016B
:105CD4000101AF6706D001010101AE51220BD8B416
:105CE40019D00101010E00010001AE6F0101AE0ED9
:105CF4000001AD6F0101010E00010001B06F01014F
:105D0400C90E0001AF6FBFC0B1F0C0C0B2F02BEC40
:105D14002FF032D001010101CA51D8B405D00101DC
:105D24000101AF51D8B42BD001010101C9A304D0A2
:105D340001010101AEA323D001010101C9AB04D0CB
:105D440001010101AEAB1BD00101010E00010001F4
:105D5400AE6F0101AE0E0001AD6F0101010E000135
:105D64000001B06F0101C90E0001AF6FBFC0B1F0F7
:105D7400C0C0B2F02BEC2FF000010001C56FBFC012
:105D84006CF0C0C06DF075EC2BF03AD0000100014E
:105D9400F051040F00010001C96F040E000100015D
:105DA400C96504D0050E00010001C95F00010001AE
:105DB400F051060D0101840EF32400010001606F0F
:105DC4000101010EF4200001616F00010001C951BD
:105DD400060D0101840EF3240001C16F0101010EBF
:105DE400F4200001C26FC1C062F0C2C063F0000EB3
:105DF40000010001656F060E0001646F81EC1FF065
:105E040000010001F02B040E0001F06508D0000130
:105E1400C16F000E00010001F06F0001C1510001CB
:105E2400C16F020E00010001FF6F0001C1510001AA
:105E3400C16F000E546E0001C1510001C16F000E0C
:105E440001010101AF6F0001C15100010001C55101
:105E54001200ADC060F0AEC061F0AFC062F0B0C07F
:105E640063F0000E00010001656F080E0001646F0D
:105E7400A7EC14F000010001615100016011D8A4E5
:105E840002D0000EF0D1B1C060F0B2C061F0000EDB
:105E940000010001636F000E0001626F000E00013B
:105EA4000001656F080E0001646FC1EC0DF0000184
:105EB40020EE01F00001AD51D9260001AE51DA22E5
:105EC400DF500001B36F0001B3A170D1ADC0D9FFA1
:105ED400AEC0DAFFDF5000010001B76F0001B36FFD
:105EE400020E00010001B96F0001B3510001B36F4C
:105EF400010E00010001BD6F0001B3510001B36F39
:105F0400020E00010001BA6F0001B3513CD100013F
:105F14000001BA51010DF35000010001AD25D96E05
:105F2400F45000010001AE21DA6EDF5000010001DF
:105F3400B86FB8C06FF00DEC20F000016FC0B5F081
:105F4400000170C0B6F00001B36F000E0001000143
:105F5400BB6F0001B3510AD100010001BB51010D17
:105F6400F35000010001B5250001B36FF4500001A6
:105F74000001B6210001B46FB3C0F6FFB4C0F7FF4F
:105F840008000001F5CFBCF0020E00010001AF25AE
:105F940000010001606F000E00010001B02100014A
:105FA400616F00010001B8C062F000010001636B81
:105FB400000E00010001656F060E0001646FDAEC4B
:105FC40012F000010001615100016011D8A402D057
:105FD400010E01D0000E00010001BE6F99D0000136
:105FE4000001BE51D8B4BFD09AEC0EF037D00001F6
:105FF4000001BE51D8B4B7D0BAEC0EF02FD00001D6
:106004000001BE51D8B4AFD03AEC0EF027D0000155
:106014000001BE51D8B4A7D07AEC0EF01FD0000115
:106024000001BE51D8B49FD05AEC0EF017D0000135
:106034000001BE51D8B497D0DAEC0EF00FD00001B5
:106044000001BE51D8B48FD0FAEC0EF007D0000195
:106054000001BE51D8B487D0E9EC25F00001B36F3C
:10606400040E00010001BD6F0001B3517CD000019A
:106074000001B78178D0110E00010001B71373D06D
:1060840000010001B7836FD000010001B78B6BD012
:1060940000010001BC51900AD8A404D00001B36FE0
:1060A400010E09D000010001BC51910AD8A409D005
:1060B4000001B36F000E00010001F26F0001B35143
:1060C40012D000010001BC51390AD8A40CD000013F
:1060D4000001BE51D8B407D01AEC0FF00009D8B4AF
:1060E40002D0010E4F1A00010001B951010DF35005
:1060F40000010001B125D96EF45000010001B22164
:10610400DA6E0001BCC0DFFF00010001B92B2BD007
:1061140000010001BC51000AD8B425D0E00AD8B46B
:10612400A6D7010AD8B4ACD7050AD8B4A4D7010AB3
:10613400D8B4AAD7130AD8B452D7010AD8B457D7B7
:106144000F0AD8B45CD7010AD8B461D7030AD8B40B
:1061540066D7060AD8B46BD7010AD8B478D7030A2D
:10616400D8B46DD795D700010001BB2B030E0001F5
:106174000001BB6105D0070E00010001B965ECD632
:1061840000010001BA2B080E00010001BA6106D01B
:1061940000010001BD51040AD8A4B9D6B1C0D9FF89
:1061A400B2C0DAFF0001B7C0DFFF38D0ADC060F085
:1061B400AEC061F083EC0FF00009D8B41ED04F508C
:1061C400D8B40CD000010001F651020AD8B415D09D
:1061D40000010001F651030AD8B40FD0ADC0A7F0F6
:1061E400AEC0A8F0AFC0A9F0B0C0AAF0B1C0ABF087
:1061F400B2C0ACF07DEC24F00ED0ADC07BF0AEC0EC
:106204007CF0AFC07DF0B0C07EF0B1C07FF0B2C012
:1062140080F0A4EC26F000010001BD6F0001000134
:10622400BD05D8B40CD000010001BD51030AD8B497
:1062340006D000010001BD51040AD8A411D0AFC09A
:1062440060F0B0C061F0ADC062F0AEC063F0000EAB
:1062540000010001656F080E0001646F81EC1FF0FE
:1062640000010001BD511200A10E0001000179617D
:10627400B9D00001000179C060F000010001616B38
:10628400000E00010001636F070E0001626FF6EC5F
:106294001EF0D89000010001603500017C6F000100
:1062A4000001613500017D6F670E00017C2500014E
:1062B4000001816F7D0E00017D210001826F0001CC
:1062C4007C6F000E00010001836F00017C5128D017
:1062D400000100018351010DF350000100018125EB
:1062E40000017C6FF45000010001822100017D6FE8
:1062F4007CC0F6FF7DC0F7FF000100018351010D52
:10630400F350000100017A25D96EF4500001000118
:106314007B21DA6E0800F5CFDFFF00010001832B3B
:10632400020E00010001836119D0000100018351B4
:10633400010DF35000010001812500017C6FF45030
:1063440000010001822100017D6F7CC0F6FF7DC049
:10635400F7FF0800F5500009D8A4BAD700010001DE
:1063640079C060F000010001616B000E00010001C2
:10637400636F070E0001626F0DEC1CF0380E000114
:1063840000016025F66E780E00016121F76E0001B0
:1063940000018351010DF350000100017A25D96EEB
:1063A400F450000100017B21DA6E0800F5CFDFFF15
:1063B40010D0000100018351010DF35000010001D0
:1063C4007A25D96EF450000100017B21DA6E000EAB
:1063D400DF6E00010001832B020E000100018365C2
:1063E400E8D799D1A00E00010001796535D0B70E28
:1063F40000010001796130D07AC06FF07BC070F089
:106404005F0E00010001792500010001696F0001A0
:1064140000016A6BFF0E6A23000E000100016C6F1D
:10642400030E00016B6FD1EC10F0B30E00010001FC
:10643400692500010001716F7C0E000100016A21D1
:106444000001726F000E00010001746F030E000161
:10645400736FCEEC11F05FD1C70E000100017965B6
:106464003DD0E10E00010001796138D07AC06FF0AF
:106474007BC070F0D89000010001793500017C6F79
:1064840000017D6B00017D37700E00017C25000149
:106494007E6FFE0E00017D2100017F6F350E00012D
:1064A4007E2500010001716F7D0E00017F21000136
:1064B400726F000E00010001746F020E0001736F11
:1064C400CEEC11F0000120EE02F000017A51D92641
:1064D40000017B51DA22000EDF6E1DD1E50E0001B2
:1064E4000001796504D1F20E000100017961FFD049
:1064F4007DD01A0E00010001792500010001696FA9
:10650400000100016A6BFF0E6A23000E0001000106
:106514006C6F030E00016B6FD1EC10F0800E000164
:106524000001692500010001816F7E0E59D01A0E09
:1065340000010001792500010001696F00010001DB
:106544006A6BFF0E6A23000E000100016C6F030EDC
:1065540000016B6FD1EC10F0380E000100016925C9
:1065640000010001816F7E0E3BD01A0E0001000174
:10657400792500010001696F000100016A6BFF0EBB
:106584006A23000E000100016C6F030E00016B6FA3
:10659400D1EC10F05C0E000100016925000100013E
:1065A400816F7E0E1DD01A0E0001000179250001B5
:1065B4000001696F000100016A6BFF0E6A23000E7F
:1065C400000100016C6F030E00016B6FD1EC10F041
:1065D400C80E00010001692500010001816F7E0ED3
:1065E400000100016A210001826F10D00001000146
:1065F400F151000AD8B4D7D7010AD8B4B6D7030AE0
:10660400D8B477D7010AD8B492D7CDD700017C6F1C
:10661400000E00010001836F00017C51020E000195
:106624000001836501D077D0000100018351010D81
:10663400F35000010001812500017C6FF45000013A
:106644000001822100017D6F7CC0F6FF7DC0F7FF51
:1066540008000001F5CF80F01AEC0FF00009D8A46F
:106664001AD02BD000017C6F300E0FD000017C6F4C
:10667400320E0BD000017C6F2E0E07D000017C6F10
:10668400250E03D000017C6F260E00010001806FEF
:1066940000017C5112D0000100018051260AD8B4B7
:1066A400EDD7010AD8B4EED7080AD8B4DBD71F0A4D
:1066B400D8B4DCD7050AD8B4DDD700010001835172
:1066C400010DF350000100017A25D96EF450000148
:1066D40000017B21DA6E000180C0DFFF00010001B0
:1066E400832B020E0001000183659ED714D07AC06B
:1066F40060F07BC061F0000E00010001636F000ECA
:106704000001626F000E00010001656F030E0001BD
:10671400646FC1EC0DF0120000010001FE51020A89
:10672400D8B43CD000010001FE51030AD8B436D0DD
:1067340042C0CAF043C0CBF00001CA1FCB1FCA4BF2
:10674400CB2BA7EC0CF00001CA510001000160251D
:106754000001CC6F0001CB51000100016121000157
:10676400CD6F0001CD51800A800F8D0ED8B4CC5D61
:10677400D8A0DED7A7EC0CF0000160C042F0000105
:1067840061C043F010EC14F0442A44C0CAF0000184
:10679400CB6BCABFCB070001CAB135D201010101DD
:1067A40081518011D8B412D080C1D9FF81C1DAFFE0
:1067B4000101DF34E836010B0001CA6F0001CA5140
:1067C40000010001CE6F0001CF6B07D0000E000165
:1067D4000001CF6F000E0001CE6F00010001CF5108
:1067E400CE11D8A4C2D100010001FE51030AD8A4DD
:1067F40025D0050105010251D8B40ED015EC0DF0D9
:10680400050105010219D8A407D00001CA6F000EC2
:1068140005010501026F0FD068EC11F005010501B7
:10682400026F05010501026772D10001CA6F000EF3
:1068340000010001FE6F0001CA5169D10001CA6F55
:10684400070E00010001D26F0001CA51A3D0C00E8F
:106854008016FC0E84163F0E9212030E961210D070
:10686400929029D0929227D0929425D0929623D0B8
:10687400929821D0929A1FD096901DD096921BD0B8
:1068840000010001D251000AD8B4EAD7010AD8B4F1
:10689400E9D7030AD8B4E8D7010AD8B4E7D7070A76
:1068A400D8B4E6D7010AD8B4E5D7030AD8B4E4D7F4
:1068B400010AD8B4E3D70001CA6F000E0001000139
:1068C400D56F0001CA515ED083B825D0010E0001F6
:1068D4000001D46F49D083BA1ED0F8D783BC1BD033
:1068E400F5D783BE18D0F2D783B415D0EFD783B6CB
:1068F40012D0ECD781BA0FD0E9D781B80CD0E6D743
:1069040081B209D0E3D781B006D0E0D781B403D0F7
:10691400DDD781A6DBD7000EDAD700010001D551FF
:10692400000AD8B4D1D7010AD8B4D5D7030AD8B449
:10693400D5D7010AD8B4D5D7070AD8B4D5D7010A10
:10694400D8B4D5D7030AD8B4D5D7010AD8B4D5D783
:106954000F0AD8B4D5D7010AD8B4D5D7030AD8B406
:10696400D5D7010AD8B4D5D700010001D451D8B481
:1069740006D0D2C07BF0D5C07CF033EC21F000010E
:106984000001D52B0B0E00010001D565C6D700010F
:106994000001D20700010001D2AF59D70501050E4D
:1069A40000010001C06F0501000E0001BF6F22EC61
:1069B4002DF000010001FE6F9BD00501050E0001C2
:1069C4000001616F0501100E0001606F000E0001EF
:1069D4000001636F000E0001626F000E00010001F0
:1069E400656F060E0001646FC1EC0DF090D00001DC
:1069F400CA6F000E00010001D36F0001CA5115D007
:106A040000010001D351010D0501020EF324D96EDA
:106A14000501050EF420DA6EDF5000010001626FFB
:106A24001EEC10F000010001D32B050E0001000143
:106A3400D365E6D70001CA6F060E00010001606F3E
:106A44000001CA51BDEC0CF005010501026F0501FE
:106A5400050E00010001616F0501030E0001606F66
:106A6400000E00010001636F000E0001626F000E52
:106A740000010001656F050E0001646FC1EC0DF0AB
:106A840046D00001CA6F030E00010001FE6F000131
:106A9400CA510001CA6F000E05010501006F000113
:106AA400CA510001CA6F800E00010001606F00012D
:106AB400CA51BDEC0CF005010501026F0501050E7C
:106AC40000010001616F0501030E0001606F000EFB
:106AD40000010001636F000E0001626F000E0001EF
:106AE4000001656F050E0001646FC1EC0DF00FD05D
:106AF40000010001FE51010AD8B409D0030AD8B438
:106B04005CD7010AD8B473D7070AD8B4BAD700013E
:106B14000001FE51D8B429D00001CA6F010E000152
:106B24000001606F0001CA510001CB6F010E00012A
:106B34000001616F0001CB510501050E0001000148
:106B4400636F0501000E0001626F0001CC6F080E37
:106B540000010001646F0001CC51F5EC1DF000014F
:106B640060C080F1000161C081F101010101835124
:106B74008211D8B412D082C1D9FF83C1DAFF0101D6
:106B8400DF34E836010B0001CA6F0001CA5100016D
:106B94000001D06F0001D16B07D0000E000100018D
:106BA400D16F000E0001D06F00010001D151D0114E
:106BB400D8A429D00001CA6F010E00010001606F42
:106BC4000001CA510001CB6F000E00010001616F8A
:106BD4000001CB510501050E00010001636F0501A1
:106BE400080E0001626F0001CC6F010E000100016C
:106BF400646F0001CC51F5EC1DF0000160C082F11E
:106C0400000161C083F1120084C0D9FF85C0DAFF9E
:106C1400DF5000010001A36F0001906F020E00011C
:106C24000001A66F000190510001906F010E000158
:106C34000001946F0001905184C0D9FF85C0DAFF30
:106C4400DF50DD0B000100019A6F88C0D9FF89C0B5
:106C5400DAFF00019AC0DFFF0001906F020E00010D
:106C64000001996F0001905190EF3AF0000100018A
:106C74009951010DF350000100018425D96EF4509F
:106C8400000100018521DA6EDF5000010001A56FCB
:106C9400A5C06FF08BEC19F000010001A46F000196
:106CA4000001A451D8B42CD000010001A651010D5B
:106CB400F350000100018825D96EF4500001000151
:106CC4008921DA6E0001A4C0DFFF00010001A62BB8
:106CD400000E00010001616F570E0001606F000E8D
:106CE40000010001636F000E0001626F000E0001DD
:106CF4000001656F030E0001646FC1EC0DF04DD20D
:106D04000001906F000E00010001956F0001905189
:106D14002F0E00010001A5653DD0540E00010001B5
:106D2400A56138D000010001A5C060F00001000198
:106D3400616B000E00010001636F0C0E0001626FB5
:106D44000DEC1CF0000100016051050A0001611105
:106D5400D8B420D000010001A5C060F000010001FA
:106D6400616B000E00010001636F0C0E0001626F85
:106D74000DEC1CF0000100016051060A00016111D4
:106D8400D8B408D00001906F010E00010001956F86
:106D94000001905195C098F00001906F020E00011F
:106DA40000019B6F0001905124D000010001985113
:106DB400D8B41CD0000100019B51010DF350000117
:106DC40000018625D96EF450000100018721DA6E96
:106DD40000010001A551DF6209D00001906F0E0E81
:106DE40000010001A56F0001905108D000010001CD
:106DF4009B2B070E000100019B65D7D70001000102
:106E0400A351220B220AD8A413D052A204D0000109
:106E14000001A3930DD086C0D9FF87C0DAFFDF50ED
:106E24000001906F000190AB03D000010001A39B0F
:106E340000010001A5C060F000010001616B000EBB
:106E440000010001636F0C0E0001626FF6EC1EF08E
:106E5400000100016151800A800F070ED8B40001BF
:106E6400605DD8A009D00001906F000E0001000100
:106E7400A26F00019051DDD000010001A3A340D016
:106E8400000E00010001636F0C0E0001626F00012F
:106E94000001A5C060F000010001616BF6EC1EF07A
:106EA400000160C069F0000161C06AF0000E0001D9
:106EB40000016C6F0C0E00016B6FD1EC10F000013F
:106EC40000016951000100018C250001906F00014F
:106ED40000016A51000100018D210001916F000140
:106EE4000001A5C060F000010001616B000E00010B
:106EF4000001636F0C0E0001626F0DEC1CF083D077
:106F040000010001A3AB40D0000E00010001636F3B
:106F14000C0E0001626F00010001A5C060F00001C9
:106F24000001616BF6EC1EF0000160C069F0000125
:106F340061C06AF0000E000100016C6F0C0E0001CC
:106F44006B6FD1EC10F000010001695100010001E8
:106F54008E250001906F000100016A5100010001BB
:106F64008F210001916F00010001A5C060F00001B4
:106F74000001616B000E00010001636F0C0E000143
:106F8400626F0DEC1CF03FD0000E00010001636F36
:106F94000C0E0001626F00010001A5C060F0000149
:106FA4000001616BF6EC1EF0000160C069F00001A5
:106FB40061C06AF0000E000100016C6F0C0E00014C
:106FC4006B6FD1EC10F00001000169510001000168
:106FD4008A250001906F000100016A51000100013F
:106FE4008B210001916F00010001A5C060F0000138
:106FF4000001616B000E00010001636F0C0E0001C3
:10700400626F0DEC1CF0000100016051000190253D
:107014000001926F00010001615100019121000102
:10702400936F92C0F6FF93C0F7FF08000001F5CFFD
:10703400A2F000010001A251D8B40DD0A2C079F091
:107044000001000E000100017B6F00019F0E000192
:107054007A6F36EC31F000010001A251D8B404D0AB
:10706400000100019F67A8D0A5C075F0CFEC29F0FE
:1070740000010001A46F00010001A451D8B44BD257
:1070840000010001A451900AD8A404D00001906F1B
:10709400010E09D000010001A451910AD8A407D01F
:1070A4000001906F000E00010001F26F49D0000151
:1070B4000001A451390AD8A42CD0020E0001000109
:1070C400862500010001606F000E00010001872188
:1070D4000001616F00010001A4C062F00001000121
:1070E400636B000E00010001656F060E0001646F02
:1070F400DAEC12F000010001615100016011D8A422
:1071040021D01AEC0FF00009D8B41CD0010E4F1A8C
:1071140019D000010001A451270AD8A413D00001FA
:107124000001A351220BD8B40DD01AEC0FF00009C2
:10713400D8B408D00001906F870E00010001A46F3D
:107144000001905100010001A651010DF35000010E
:1071540000018825D96EF450000100018921DA6EFE
:107164000001A4C0DFFF00010001A62B000E0001F6
:107174000001616F570E0001606F000E00010001F5
:10718400636F000E0001626F000E00010001656F65
:10719400030E0001646FC1EC0DF084C0D9FF85C0FB
:1071A400DAFFDF50526E84C0D9FF85C0DAFFDF50AA
:1071B400000100019A6FAFD1000100019851D8B4C9
:1071C40076D00001906F000E000100019C6F000159
:1071D400905159D00001906F000E000100019D6F85
:1071E4000001905139D0000100019C51010D0101B1
:1071F400BE0EF324D96E0101010EF420DA6E0001F3
:1072040000019D51010D00019F0EF324E16E000168
:10721400000EF420E26EE750DF621BD00101010E84
:1072240000010001616F0101BE0E0001606F000EDC
:1072340000010001636F000E0001626F000E000187
:107244000001656F030E0001646FC1EC0DF0020EC6
:10725400BCD1000100019D2B030E000100019D61C2
:107264000FD0000100019D51010D00019F0EF32478
:10727400D96E0001000EF420DA6EDF50D8A4B3D723
:10728400000100019C2B030E000100019C610FD042
:10729400000100019C51010D0101BE0EF324D96EC1
:1072A4000101010EF420DA6EDF50D8A493D7000157
:1072B400906F030E00010001946F000190510001D2
:1072C400906F000E000100019E6F00019051EBD001
:1072D400000100019E51010D00019F0EF324D96E9F
:1072E4000001000EF420DA6EDF5000010001A46FEB
:1072F400C7D05750D8B4D4D07F0E00010001616FBD
:10730400F60E0001606F000157C062F00001000139
:10731400636B000E00010001656F040E0001646FD1
:10732400DAEC12F0000160C096F0000161C097F041
:107334000001000197519611D8B4B2D0060E000195
:107344000001A661ADD000010001A651010DF3506A
:10735400000100018825D96EF45000010001892143
:10736400DA6E2A0EDF6E00010001A62BF60E000174
:10737400906F7F0E916F0001901F911F904B912B86
:10738400000100019651000190270001000197516E
:1073940000019123450E00019025F66E780E91218F
:1073A400F76E00010001A651010DF3500001000128
:1073B4008825D96EF450000100018921DA6E080095
:1073C400F5CFDFFF2CD057500B0AD8A469D0060E96
:1073D40000010001A66164D000010001A651010D65
:1073E400F350000100018825D96EF450000100011A
:1073F4008921DA6E2A0EDF6E00010001A62B00013E
:107404000001A651010DF350000100018825D96E39
:10741400F450000100018921DA6E130EDF6E0001C1
:107424000001A62B00010001A651010DF35000013B
:1074340000018825D96EF450000100018921DA6E1B
:1074440058C0DFFF19D0000100019A8329D0000140
:1074540000019A8B25D000010001A651010DF350C3
:10746400000100018825D96EF45000010001892132
:10747400DA6E0001A4C0DFFF00010001A62B10D0CA
:1074840000010001A451E10AD8B4DDD7040AD8B43C
:10749400DED7160AD8B42DD7070AD8B494D7DBD7C9
:1074A400000100019E2B030E000100019E6114D017
:1074B400000100019E51010D00019F0EF324D96EBD
:1074C4000001000EF420DA6EDF50D8B405D0070EA8
:1074D40000010001A665FCD6000E00010001706FDA
:1074E400570E00016F6F0001000E00010001726F62
:1074F40000019F0E0001716F000E00010001746F06
:10750400030E0001736FCEEC11F084C0D9FF85C067
:10751400DAFFDF50526E00010001992B080E0001C2
:107524000001996106D0070E00010001A66538EF3D
:1075340036F0020E00010001A66521D00101010E02
:1075440000010001706F0101BE0E00016F6F000E9B
:1075540000010001726F570E0001716F000E0001EF
:107564000001746F030E0001736FCEEC11F088C03C
:10757400D9FF89C0DAFF00019AC0DFFF23D00101DF
:10758400010E00010001616F0101BE0E0001606F78
:10759400000E00010001636F000E0001626F000E17
:1075A40000010001656F030E0001646FC1EC0DF072
:1075B40084C0D9FF85C0DAFF88C0E1FF89C0E2FF3B
:1075C400DFCFE7FF00010001945112000D01020317
:1075D4000405060708090A1624000E0E0E0E0E0EE8
:1075E4000E0E0B2F54180E0E0E41420E0E0E235F7C
:1075F400550C0E0E0E4D4E0E0E0E175E5619252608
:1076040027282B2C2D2E225D573031323334373836
:10761400393A3B5C583C3D3E3F4043444546475B1A
:107624005948494A4B4C4F505152535A2F3B3C3DB9
:107634003E3F40414243442E353A000000000000E2
:1076440000004531301E0000000000000000272D1E
:107654002A1F20212200002324252634141A09136A
:107664000A00000D0F181C33041516170729650BA3
:1076740011080C121D1B0619052B280E103637385D
:10768400E0E3F0E12CE2E62CE5F0E7E42F3B3C3DBF
:107694003E3F404142434431353A0000000000007F
:1076A4000000452E301E00000000000000002738B6
:1076B400391F2021220000232425262D3436371398
:1076C4001C0000090A06150F041208180C29650786
:1076D4000B17111633140D0E1B2B2805101A191D28
:1076E400E0E3F0E12AE2E62CE5F0E7E4303B3C3D60
:1076F4003E3F40414243442E893A000000000000CE
:107704000000452F321E0000000000000000272D5D
:10771400391F20212200002324252634141A081599
:107724001700001C180C1213041607090A29650B0C
:107734000D0E0F331D1B0619052B28111036373873
:10774400E0E3F0E12AE2E62CE5F0E7E4303B3C3DFF
:107754003E3F40414243442D893A0000000000006E
:107764000000452F321E00000000000000002734F6
:107774002E1F2021220000232425262A141A08154E
:107784001700001C180C1213041607090A29650BAC
:107794000D0E0F331D1B0619052B28111036373813
:1077A400E0E3F0E158E2E62CE5F0E7E42F3B3C3D72
:1077B4003E3F40414243442E353A00000000000061
:1077C40000004531301E0000000000000000272D9D
:1077D400391F20212200002324252634141A0815D9
:1077E4001700001C180C1213041607090A29650B4C
:1077F4000D0E0F331D1B0619052B281110363738B3
:10780400E0E3F0E12AE2E62CE5F0E7E40000000022
:107814000000000000000000005500FB0067540059
:10782400005F606156005C5D5E5700595A5B28003A
:107834006200630000040C1808121CFA7F5F7FBF0B
:107844007D0A1D0705E97D490000F80000F60000E7
:10785400F70000F90000FA0000FE0000FC00000040
:1078640000007F0000810000480000E04C00FD00A3
:107874000000000000000000000000000000000004
:10788400000000000000000000800000470000E04D
:10789400E11DE01E000000000000000000000000E8
:1078A40000000000000000000000000000E02700CD
:1078B4004600004C0000E01F00E02000E02100E052
:1078C4002200000000000000E02300E0E150E1524B
:1078D40000E0E14F530000E01400E01A004B000008
:1078E400E01500E01700000000000000E04A00E09E
:1078F4005000520000E04F00E04D00E00400E016AC
:10790400004E0000E00900E00A00290000390000F0
:107914004A00005000005100004F00004D0000E0FC
:107924001D00E01B00E00600E019009100002B00A0
:1079340000280000900000E15000E15100E14F00F8
:10794400E14D000000000000000000000000000005
:107954000000000000000000000000000000000023
:107964000000000000000000000000000000000013
:107974000000000000000000000000000000000003
:1079840000000000000000000000000000000000F3
:1079940000000000000000B69AB5B4B300002A311C
:1079A400383F4604030201050000070E151C23AEF0
:1079B4006993A4B200004D545BCD62000000000046
:1079C40000000000000000000000000000000000B3
:1079D40000000000000000000000000000000000A3
:1079E4000000000000000000000000ACA9A6A2B046
:1079F4000000307A3EC84CABA8A5A1AF00000D141E
:107A04001B2229ADAAA7A3B10000535A61CE680076
:107A140000000000000000000000CA000000000098
:107A24000000000000000000000000000000000052
:107A34000000CD000000000000000000000000CEA7
:107A440008160C0F000039170A18CD0310190B1271
:107A54000000241A0902C8CE2511262700002E137F
:107A64002028EC0000000000000000000000CA0014
:107A7400000000000000000000000000CC00000036
:107A84000000000000000000EDF1E6E70000EAEB72
:107A94000000006A043A7F3C0000475D505E4844A1
:107AA400011D812F000063604F4BC86CC93D326BD0
:107AB400000049594A67ECE800000000000000009B
:107AC4000000CB000000000000000000000000E9FE
:107AD400CC0000000000000000000000EDF1E6E72B
:107AE4000000EAEB000000CE4E5C52550000361E4A
:107AF4003B2B6D96565F515800002C0521837ACE9E
:107B04006457656600001F342D406ED300000000EA
:107B14000000000000000000000000000000000061
:107B2400000000D4D7000000000000000000DE00C8
:107B340000000000000000000000DD000000000064
:107B4400000000000000D100000000000000000060
:107B54000000000000DB0000000000000000E0D393
:107B64000000000000000000000000000000000011
:107B740000000000000000D400000000000000002D
:107B84000000DE0000000000000000000000DF0034
:107B94000000B300000000000000D2000046D6D56B
:107BA400000000D9D8DC000000000000000000DA6A
:107BB40000000000000000000000000000000000C1
:107BC40000000000000000000000000000000000B1
:107BD40000000000000000000000000000000000A1
:107BE400000000393B0C2483000009210A013C16E3
:107BF4001A08192F000044020310C82B3A1E0F1D47
:107C040000001118CDCE7A00000000000000000032
:107C1400000000EE00000000000000000000000072
:107C24000000000000000000000000000000000050
:107C3400000000000000002513EC7F2800004F51D5
:107C440050CC8E1F208136260000CA5D9656906D5A
:107C54006E1234270000575EEFF086E80000000043
:107C64000000000000000000000000000000000010
:107C7400000000E900000000000000000000000017
:107C84000000000000000000000000645952636717
:107C94000000040B2E2D3D5C604E5F65000005174F
:107CA400C92C3271745855660000406B6ACB6C0461
:107CB4001111040E18041718040C000C11110C0EE9
:107CC400180C1718181111180E1818171808111174
:107CD400080E0C081718080C00121111120E1812B5
:107CE40017181218000600000900000D0000140007
:107CF4000005010906A101050719E029E71500257A
:107D04000175019508810295017508810395057532
:107D1400010508190129059102950175039103953F
:107D2400067508150026FF000507190029FF8100C4
:107D3400C011112D00F300F400E13836003700E1E2
:107D440036E1372F003000E130E13234002E002DCF
:107D5400001E0038003200E1278700E136E137E1F8
:107D640038890000000E001600170011000B0010E7
:107D7400001C0015001A0013000A001D000700056E
:107D8400001B001B0E1B171B1C1B1A1A1C19000FAF
:107D940000E0E1E3E2E6E5E4E0E1E29190E5E4E03D
:107DA400E1E39190E5E4E1E0E3E2E6E4E5E1E0E249
:107DB4009190E4E5E1E0E39190E4E52A0345007362
:107DC40000720069006C006C00650020004E0065C4
:107DD40000770020004B006500790062006F0061AD
:107DE400007200640009022900010100A0320904A4
:107DF40000000203010100092111010001224000D9
:107E040007058103080001070501030800010612A4
:107E1400131C150C0A0B172C1F271E20362C1F278A
:107E24001E212C0816150C0F0F082C0C11063728D0
:107E3400091F2C002F0000300000E12F00E130006A
:107E4400E2E126E2E127380000380000383838360D
:107E54000000370000E135002F00003000002F0043
:107E6400003000002F00003000003800003800000F
:107E7400383838360000370000E135002F00003074
:107E840000001D2F001D30002F00003000001D38A1
:107E9400003800001D3700360000370000E13500CF
:107EA400062800000000060D28000000060D10043E
:107EB4000628162800000000160D28000000160DE4
:107EC400100406282F00003000002F0000300000AE
:107ED4002F000030000038000038000038383836F1
:107EE4000000370000E13500151210042800110CC1
:107EF4000612280010171C13082817151211280041
:107F040016170C060E281306280000100406280075
:107F14001E272604281E27260528042D1613281696
:107F24002D1613280F28000006280000152800002D
:107F34000F2D1128062D0628152D1628120909289B
:107F44000816150C0F0F082C11081A2C0E081C0506
:107F54001204150728150819372C001A0345007355
:107F640000720069006C006C006500200049006E1E
:107F74000063002E00181628000018162D07281874
:107F8400162D06280D132800000D132D1128072780
:107F94002800071E1F28071F212807202328072140
:107FA400252810162800000417120E280A12120A97
:107FB400280413130F281201000200000008D8043B
:107FC40050F50100010200018B00008A00008800C6
:107FD40000350000190815372C0009202C00092150
:107FE4002C0009222C0009232C0009242C0009252B
:0C7FF4002C000E16170B040309040000FB
:020000040020DA
:08000000FFFFFFFFFFFFFFFF00
:020000040030CA
:0E000000330E3F1EFF8181FF0FC00FE00F4047
:0200000400F00A
:080000000000000100040000F3
:00000001FF
